******************************************************************************
               TMS320C6x Linker PC v7.4.24                     
******************************************************************************
>> Linked Wed Feb 13 17:12:05 2019

OUTPUT FILE NAME:   <GE.out>
ENTRY POINT SYMBOL: "_c_int00"  address: 0c081920


MEMORY CONFIGURATION

         name            origin    length      used     unused   attr    fill
----------------------  --------  ---------  --------  --------  ----  --------
  VECTORS               00800000   00000200  00000200  00000000  RWIX
  LL2_RW_DATA           00800200   0003fe00  00038180  00007c80  RWIX
  SL2                   0c000000   00200000  0008710b  00178ef5  RWIX
  DDR3_CODE             80000000   01000000  00000000  01000000  RWIX
  DDR3_R_DATA           81000000   01000000  00000000  01000000  RWIX
  DDR3_RW_DATA          82000000   06000000  00346000  05cba000  RWIX


SEGMENT ALLOCATION MAP

run origin  load origin   length   init length attrs members
----------  ----------- ---------- ----------- ----- -------
00800000    00800000    00000200   00000200    r-x
  00800000    00800000    00000200   00000200    r-x vecs
00800200    00800200    00034000   00000000    rw-
  00800200    00800200    00034000   00000000    rw- PacketData:buffer_LL2
00834200    00834200    00002320   00001320    rw-
  00834200    00834200    00001320   00001320    rw- .far
  00835520    00835520    00001000   00000000    rw- .stack
00836540    00836540    00001400   00000000    rw-
  00836540    00836540    00000c00   00000000    rw- QMSS_Data:Descriptor_LL2
  00837140    00837140    00000800   00000000    rw- .sysmem
00837940    00837940    00000921   00000921    rw-
  00837940    00837940    000007d4   000007d4    rw- .fardata
  00838114    00838114    0000014d   0000014d    rw- .neardata
00838264    00838264    0000001c   00000000    rw-
  00838264    00838264    0000001c   00000000    rw- .bss
00838280    00838280    00000120   00000000    rw-
  00838280    00838280    00000120   00000000    rw- .cio
0c000000    0c000000    00068000   00000000    rw-
  0c000000    0c000000    00068000   00000000    rw- PacketData:buffer_SL2
0c068000    0c068000    0001de4b   0001de4b    r-x
  0c068000    0c068000    00019f40   00019f40    r-x .text
  0c081f40    0c081f40    00003f0b   00003f0b    r-- .const
0c085e4c    0c085e4c    00000010   00000010    r--
  0c085e4c    0c085e4c    00000010   00000010    r-- .switch
0c085e80    0c085e80    00000c00   00000000    rw-
  0c085e80    0c085e80    00000c00   00000000    rw- QMSS_Data:Descriptor_SL2
0c086a80    0c086a80    000006b0   000006b0    r--
  0c086a80    0c086a80    000006b0   000006b0    r-- .cinit
82000000    82000000    00346000   00000000    rw-
  82000000    82000000    00340000   00000000    rw- PacketData:buffer_DDR
  82340000    82340000    00006000   00000000    rw- QMSS_Data:Descriptor_DDR


SECTION ALLOCATION MAP

 output                                  attributes/
section   page    origin      length       input sections
--------  ----  ----------  ----------   ----------------
vecs       0    00800000    00000200     
                  00800000    00000200     GE_vectors.obj (vecs)

PacketData:buffer_LL2 
*          0    00800200    00034000     UNINITIALIZED
                  00800200    00034000     GE_PktDMA_Init.obj (PacketData:buffer_LL2)

.far       0    00834200    00001320     
                  00834200    00000c00     GE_2DSP_Test.obj (.far) [fill = 0]
                  00834e00    00000240     KeyStone_GE_Init_drv.obj (.far) [fill = 0]
                  00835040    00000208     GE_PktDMA_Init.obj (.far) [fill = 0]
                  00835248    00000140     rts6600_elf.lib : defs.obj (.far) [fill = 0]
                  00835388    00000100     GE_Test.obj (.far) [fill = 0]
                  00835488    0000006c     KeyStone_common.obj (.far) [fill = 0]
                  008354f4    00000004     --HOLE--
                  008354f8    00000010     KeyStone_DDR_Init.obj (.far:Core_MPAX)
                  00835508    00000010     KeyStone_common.obj (.far:Core_MPAX)
                  00835518    00000008     rts6600_elf.lib : trgdrv.obj (.far) [fill = 0]

.stack     0    00835520    00001000     UNINITIALIZED
                  00835520    00000008     rts6600_elf.lib : boot.obj (.stack)
                  00835528    00000ff8     --HOLE--

QMSS_Data:Descriptor_LL2 
*          0    00836540    00000c00     UNINITIALIZED
                  00836540    00000c00     GE_PktDMA_Init.obj (QMSS_Data:Descriptor_LL2)

.sysmem    0    00837140    00000800     UNINITIALIZED
                  00837140    00000008     rts6600_elf.lib : memory.obj (.sysmem)
                  00837148    000007f8     --HOLE--

.fardata   0    00837940    000007d4     
                  00837940    000001e0     rts6600_elf.lib : defs.obj (.fardata:_ftable)
                  00837b20    00000120     GE_PktDMA_Init.obj (.fardata:freeHostQueueCfgTable)
                  00837c40    000000a0     rts6600_elf.lib : lowlev.obj (.fardata:_stream)
                  00837ce0    00000078                     : lowlev.obj (.fardata:_device)
                  00837d58    00000070     GE_PktDMA_Init.obj (.fardata:flowCfgTable)
                  00837dc8    00000048     GE_PktDMA_Init.obj (.fardata:descMemRegionsCfg)
                  00837e10    00000040     KeyStone_common.obj (.fardata:gstruMpuAddrRange)
                  00837e50    00000030     GE_PktDMA_Init.obj (.fardata:FDQ_str)
                  00837e80    00000028     KeyStone_common.obj (.fardata:gpEDMA_TC_regs)
                  00837ea8    00000024     KeyStone_common.obj (.fardata:gpTimerRegs)
                  00837ecc    00000004     rts6600_elf.lib : defs.obj (.fardata)
                  00837ed0    00000024     KeyStone_common.obj (.fardata:input_clk_str)
                  00837ef4    00000004     --HOLE--
                  00837ef8    00000024     KeyStone_common.obj (.fardata:internal_exception_str)
                  00837f1c    00000004     --HOLE--
                  00837f20    00000020     KeyStone_common.obj (.fardata:boot_mode_str)
                  00837f40    00000020     KeyStone_common.obj (.fardata:bus_err_stat_str)
                  00837f60    00000020     KeyStone_common.obj (.fardata:gCIC_EXC_EN_MASK)
                  00837f80    00000020     KeyStone_common.obj (.fardata:gpMPU_regs)
                  00837fa0    00000020     GE_loopback_Test.obj (.fardata:message_src_dest)
                  00837fc0    00000020     GE_loopback_Test.obj (.fardata:multiPortTest)
                  00837fe0    00000018     GE_Test.obj (.fardata:GE_mode_str)
                  00837ff8    00000018     KeyStone_common.obj (.fardata:Peri_MPU_err_type_str)
                  00838010    00000018     GE_PktDMA_Init.obj (.fardata:flow_str)
                  00838028    00000018     GE_2DSP_Test.obj (.fardata:test_2DSP_cfg)
                  00838040    00000014     KeyStone_common.obj (.fardata:device_type_str)
                  00838054    00000004     --HOLE--
                  00838058    00000010     GE_Test.obj (.fardata:Dest_MAC_address)
                  00838068    00000010     GE_Test.obj (.fardata:Source_MAC_address)
                  00838078    0000000c     GE_debug.obj (.fardata:GE_speed_str)
                  00838084    00000004     --HOLE--
                  00838088    0000000c     KeyStone_common.obj (.fardata:gpEDMA_CC_regs)
                  00838094    0000000c     rts6600_elf.lib : exit.obj (.fardata)
                  008380a0    0000000c                     : memory.obj (.fardata)
                  008380ac    00000004     --HOLE--
                  008380b0    00000008     GE_debug.obj (.fardata:GE_duplex_str)
                  008380b8    00000008     KeyStone_common.obj (.fardata:Ns_str)
                  008380c0    00000008     KeyStone_common.obj (.fardata:endian_str)
                  008380c8    00000008     KeyStone_GE_Init_drv.obj (.fardata:gpCPSW_port_regs)
                  008380d0    00000008     KeyStone_GE_Init_drv.obj (.fardata:gpMAC_regs)
                  008380d8    00000008     KeyStone_Navigator_init_drv.obj (.fardata:gpQM_PDSP_Cmd)
                  008380e0    00000008     KeyStone_Navigator_init_drv.obj (.fardata:gpQM_PDSP_CtrlRegs)
                  008380e8    00000008     KeyStone_Navigator_init_drv.obj (.fardata:gpQM_PDSP_IRAM)
                  008380f0    00000008     KeyStone_GE_Init_drv.obj (.fardata:gpSGMII_regs)
                  008380f8    00000008     KeyStone_GE_Init_drv.obj (.fardata:gpStats_regs)
                  00838100    00000008     GE_Test.obj (.fardata:port_connect)
                  00838108    00000008     rts6600_elf.lib : _lock.obj (.fardata)
                  00838110    00000004     KeyStone_GE_Init_drv.obj (.fardata:STATS_EN)

.neardata 
*          0    00838114    0000014d     
                  00838114    000000bc     KeyStone_common.obj (.neardata)
                  008381d0    00000064     KeyStone_Navigator_init_drv.obj (.neardata)
                  00838234    0000000c     GE_2DSP_Test.obj (.neardata)
                  00838240    0000000c     GE_Interrupts.obj (.neardata)
                  0083824c    0000000c     KeyStone_GE_Init_drv.obj (.neardata)
                  00838258    00000008     GE_Test.obj (.neardata)
                  00838260    00000001     GE_loopback_Test.obj (.neardata)

.rodata    0    00838261    00000000     UNINITIALIZED

.bss       0    00838264    0000001c     UNINITIALIZED
                  00838264    00000014     GE_PktDMA_Init.obj (.bss)
                  00838278    00000004     GE_Interrupts.obj (.bss)
                  0083827c    00000004     KeyStone_GE_Init_drv.obj (.bss)

.cio       0    00838280    00000120     UNINITIALIZED
                  00838280    00000120     rts6600_elf.lib : trgmsg.obj (.cio)

PacketData:buffer_SL2 
*          0    0c000000    00068000     UNINITIALIZED
                  0c000000    00068000     GE_PktDMA_Init.obj (PacketData:buffer_SL2)

.text      0    0c068000    00019f40     
                  0c068000    00005c20     KeyStone_common.obj (.text)
                  0c06dc20    000029c0     KeyStone_DDR_Init.obj (.text)
                  0c0705e0    000023a0     KeyStone_GE_Init_drv.obj (.text)
                  0c072980    00001a80     KeyStone_Navigator_init_drv.obj (.text)
                  0c074400    00001740     common_test.obj (.text)
                  0c075b40    000012a0     GE_debug.obj (.text)
                  0c076de0    00000e60     GE_loopback_Test.obj (.text)
                  0c077c40    00000d40     GE_Test.obj (.text)
                  0c078980    00000aa0     GE_2DSP_Test.obj (.text)
                  0c079420    00000a00     Keystone_Serdes_init.obj (.text)
                  0c079e20    00000620     GE_Interrupts.obj (.text:retain)
                  0c07a440    00000600     KeyStone_common.obj (.text:retain)
                  0c07aa40    000005c0     rts6600_elf.lib : divd.obj (.text:__c6xabi_divd)
                  0c07b000    000005c0                     : _printfi.obj (.text:_getarg_diouxp)
                  0c07b5c0    00000540     GE_PktDMA_Init.obj (.text)
                  0c07bb00    00000520     rts6600_elf.lib : _printfi.obj (.text:_setfield)
                  0c07c020    000004a0     GE_Interrupts.obj (.text)
                  0c07c4c0    00000460     rts6600_elf.lib : _printfi.obj (.text:_printfi)
                  0c07c920    00000440     KeyStone_common.obj (.text:Core_MPAX)
                  0c07cd60    000003a0     rts6600_elf.lib : fputs.obj (.text:fputs)
                  0c07d100    00000340                     : _printfi.obj (.text:fcvt)
                  0c07d440    00000320                     : _printfi.obj (.text:_pproc_fge)
                  0c07d760    00000320                     : _printfi.obj (.text:ecvt)
                  0c07da80    000002e0                     : _printfi.obj (.text:_pproc_fwp)
                  0c07dd60    000002c0                     : _printfi.obj (.text:_pconv_e)
                  0c07e020    00000280                     : divf.obj (.text:__c6xabi_divf)
                  0c07e2a0    00000280                     : memory.obj (.text:free)
                  0c07e520    00000240                     : imath64.obj (.text:__c6xabi_divull)
                  0c07e760    00000240                     : _printfi.obj (.text:_pproc_diouxp)
                  0c07e9a0    00000220                     : _printfi.obj (.text:_pproc_str)
                  0c07ebc0    00000220                     : fputc.obj (.text:fputc)
                  0c07ede0    00000200                     : _printfi.obj (.text:_pconv_g)
                  0c07efe0    00000200                     : setvbuf.obj (.text:setvbuf)
                  0c07f1e0    000001c0                     : _printfi.obj (.text:_mcpy)
                  0c07f3a0    000001a0                     : trgdrv.obj (.text:HOSTrename)
                  0c07f540    000001a0                     : imath40.obj (.text:__c6xabi_divul)
                  0c07f6e0    00000180                     : copy_decompress_rle.obj (.text:__TI_decompress_rle_core)
                  0c07f860    00000180                     : memory.obj (.text:malloc)
                  0c07f9e0    00000140                     : _printfi.obj (.text:_pproc_fflags)
                  0c07fb20    00000140                     : lowlev.obj (.text:getdevice)
                  0c07fc60    00000120                     : fclose.obj (.text:_closefile)
                  0c07fd80    00000120                     : _printfi.obj (.text:_ltostr)
                  0c07fea0    00000120                     : fseek.obj (.text:fseek)
                  0c07ffc0    00000100                     : trgdrv.obj (.text:HOSTlseek)
                  0c0800c0    00000100                     : autoinit.obj (.text:_auto_init_elf)
                  0c0801c0    00000100                     : _io_perm.obj (.text:_wrt_ok)
                  0c0802c0    00000100                     : cpy_tbl.obj (.text:copy_in)
                  0c0803c0    000000e0                     : trgdrv.obj (.text:HOSTopen)
                  0c0804a0    000000e0                     : trgdrv.obj (.text:HOSTread)
                  0c080580    000000e0                     : _printfi.obj (.text:_div)
                  0c080660    000000e0                     : atoi.obj (.text:atoi)
                  0c080740    000000e0                     : lowlev.obj (.text:close)
                  0c080820    000000e0                     : copy_zero_init.obj (.text:decompress:ZI:__TI_zero_init)
                  0c080900    000000e0                     : ltoa.obj (.text:ltoa)
                  0c0809e0    000000e0                     : memset.obj (.text:memset)
                  0c080ac0    000000e0                     : printf.obj (.text:printf)
                  0c080ba0    000000c0                     : trgdrv.obj (.text:HOSTunlink)
                  0c080c60    000000c0                     : trgdrv.obj (.text:HOSTwrite)
                  0c080d20    000000c0                     : divu.obj (.text:__divu)
                  0c080de0    000000c0                     : fflush.obj (.text:_doflush)
                  0c080ea0    000000c0                     : exit.obj (.text:exit)
                  0c080f60    000000c0                     : tls.obj (.text:tls:init:__TI_tls_init)
                  0c081020    000000a0                     : trgdrv.obj (.text:HOSTclose)
                  0c0810c0    000000a0                     : fopen.obj (.text:_cleanup)
                  0c081160    000000a0                     : _printfi.obj (.text:_ecpy)
                  0c081200    000000a0                     : _printfi.obj (.text:_fcpy)
                  0c0812a0    000000a0                     : memory.obj (.text:_minit)
                  0c081340    000000a0                     : _printfi.obj (.text:_pconv_f)
                  0c0813e0    000000a0                     : lowlev.obj (.text:finddevice)
                  0c081480    000000a0                     : lowlev.obj (.text:lseek)
                  0c081520    000000a0                     : memcpy64.obj (.text:memcpy)
                  0c0815c0    000000a0                     : memory.obj (.text:minsert)
                  0c081660    000000a0                     : memory.obj (.text:mremove)
                  0c081700    000000a0                     : lowlev.obj (.text:write)
                  0c0817a0    00000080                     : fixdu.obj (.text:__c6xabi_fixdu)
                  0c081820    00000080                     : fixfu.obj (.text:__c6xabi_fixfu)
                  0c0818a0    00000080                     : llshift.obj (.text:__c6xabi_llshl)
                  0c081920    00000080                     : boot.obj (.text:_c_int00)
                  0c0819a0    00000080                     : trgmsg.obj (.text:readmsg)
                  0c081a20    00000080                     : lowlev.obj (.text:unlink)
                  0c081aa0    00000060                     : cpp_init.obj (.text:__TI_cpp_init)
                  0c081b00    00000060                     : frcmpyd_div.obj (.text:__c6xabi_frcmpyd_div)
                  0c081b60    00000060                     : llshift.obj (.text:__c6xabi_llshru)
                  0c081bc0    00000060                     : imath64.obj (.text:_subcull)
                  0c081c20    00000060                     : memccpy.obj (.text:memccpy)
                  0c081c80    00000060                     : trgmsg.obj (.text:writemsg)
                  0c081ce0    00000040     GE_vectors.obj (.text)
                  0c081d20    00000040     rts6600_elf.lib : isinf.obj (.text:__c6xabi_isinf)
                  0c081d60    00000040                     : _printfi.obj (.text:__c6xabi_isnan)
                  0c081da0    00000040                     : strasg.obj (.text:__strasgi_64plus)
                  0c081de0    00000040                     : args_main.obj (.text:_args_main)
                  0c081e20    00000040                     : fputs.obj (.text:puts)
                  0c081e60    00000020                     : negll.obj (.text:__c6xabi_negll)
                  0c081e80    00000020                     : _lock.obj (.text:_nop)
                  0c081ea0    00000020                     : printf.obj (.text:_outc)
                  0c081ec0    00000020                     : printf.obj (.text:_outs)
                  0c081ee0    00000020                     : exit.obj (.text:abort)
                  0c081f00    00000020                     : copy_decompress_none.obj (.text:decompress:none:__TI_decompress_none)
                  0c081f20    00000020                     : copy_decompress_rle.obj (.text:decompress:rle24:__TI_decompress_rle24)

.const     0    0c081f40    00003f0b     
                  0c081f40    00001a2c     KeyStone_common.obj (.const:.string)
                  0c08396c    000006a4     GE_debug.obj (.const:.string)
                  0c084010    00000640     GE_PktDMA_Init.obj (.const:acc32_le)
                  0c084650    00000630     GE_PktDMA_Init.obj (.const:acc16_le)
                  0c084c80    00000504     common_test.obj (.const:.string)
                  0c085184    00000308     GE_Test.obj (.const:.string)
                  0c08548c    00000248     GE_PktDMA_Init.obj (.const:.string)
                  0c0856d4    00000248     GE_loopback_Test.obj (.const:.string)
                  0c08591c    00000154     KeyStone_Navigator_init_drv.obj (.const:.string)
                  0c085a70    00000108     GE_Interrupts.obj (.const:.string)
                  0c085b78    00000101     rts6600_elf.lib : ctype.obj (.const:.string:_ctypes_)
                  0c085c79    00000002                     : fputs.obj (.const:.string)
                  0c085c7b    00000001     --HOLE-- [fill = 0]
                  0c085c7c    000000ac     GE_2DSP_Test.obj (.const:.string)
                  0c085d28    00000070     KeyStone_DDR_Init.obj (.const:.string)
                  0c085d98    00000054     KeyStone_GE_Init_drv.obj (.const:.string)
                  0c085dec    00000004     --HOLE-- [fill = 0]
                  0c085df0    00000038     common_test.obj (.const:$P$T0$1)
                  0c085e28    00000023     rts6600_elf.lib : _printfi.obj (.const:.string)

.switch    0    0c085e4c    00000010     
                  0c085e4c    00000010     GE_Test.obj (.switch:main)

QMSS_Data:Descriptor_SL2 
*          0    0c085e80    00000c00     UNINITIALIZED
                  0c085e80    00000c00     GE_PktDMA_Init.obj (QMSS_Data:Descriptor_SL2)

.cinit     0    0c086a80    000006b0     
                  0c086a80    000004af     (.cinit..fardata.load) [load image, compression = rle]
                  0c086f2f    00000001     --HOLE-- [fill = 0]
                  0c086f30    00000141     (.cinit..neardata.load) [load image, compression = rle]
                  0c087071    00000003     --HOLE-- [fill = 0]
                  0c087074    00000027     (.cinit..far.load) [load image, compression = rle]
                  0c08709b    00000001     --HOLE-- [fill = 0]
                  0c08709c    0000000c     (__TI_handler_table)
                  0c0870a8    00000008     (.cinit..bss.load) [load image, compression = zero_init]
                  0c0870b0    00000008     (.cinit.PacketData:buffer_DDR.load) [load image, compression = zero_init]
                  0c0870b8    00000008     (.cinit.PacketData:buffer_LL2.load) [load image, compression = zero_init]
                  0c0870c0    00000008     (.cinit.PacketData:buffer_SL2.load) [load image, compression = zero_init]
                  0c0870c8    00000008     (.cinit.QMSS_Data:Descriptor_DDR.load) [load image, compression = zero_init]
                  0c0870d0    00000008     (.cinit.QMSS_Data:Descriptor_LL2.load) [load image, compression = zero_init]
                  0c0870d8    00000008     (.cinit.QMSS_Data:Descriptor_SL2.load) [load image, compression = zero_init]
                  0c0870e0    00000050     (__TI_cinit_table)

PacketData:buffer_DDR 
*          0    82000000    00340000     UNINITIALIZED
                  82000000    00340000     GE_PktDMA_Init.obj (PacketData:buffer_DDR)

QMSS_Data:Descriptor_DDR 
*          0    82340000    00006000     UNINITIALIZED
                  82340000    00006000     GE_PktDMA_Init.obj (QMSS_Data:Descriptor_DDR)


LINKER GENERATED COPY TABLES

__TI_cinit_table @ 0c0870e0 records: 10, size/record: 8, table size: 80
	.fardata: load addr=0c086a80, load size=000004af bytes, run addr=00837940, run size=000007d4 bytes, compression=rle
	.neardata: load addr=0c086f30, load size=00000141 bytes, run addr=00838114, run size=0000014d bytes, compression=rle
	.far: load addr=0c087074, load size=00000027 bytes, run addr=00834200, run size=00001320 bytes, compression=rle
	.bss: load addr=0c0870a8, load size=00000008 bytes, run addr=00838264, run size=0000001c bytes, compression=zero_init
	PacketData:buffer_DDR: load addr=0c0870b0, load size=00000008 bytes, run addr=82000000, run size=00340000 bytes, compression=zero_init
	PacketData:buffer_LL2: load addr=0c0870b8, load size=00000008 bytes, run addr=00800200, run size=00034000 bytes, compression=zero_init
	PacketData:buffer_SL2: load addr=0c0870c0, load size=00000008 bytes, run addr=0c000000, run size=00068000 bytes, compression=zero_init
	QMSS_Data:Descriptor_DDR: load addr=0c0870c8, load size=00000008 bytes, run addr=82340000, run size=00006000 bytes, compression=zero_init
	QMSS_Data:Descriptor_LL2: load addr=0c0870d0, load size=00000008 bytes, run addr=00836540, run size=00000c00 bytes, compression=zero_init
	QMSS_Data:Descriptor_SL2: load addr=0c0870d8, load size=00000008 bytes, run addr=0c085e80, run size=00000c00 bytes, compression=zero_init


LINKER GENERATED HANDLER TABLE

__TI_handler_table @ 0c08709c records: 3, size/record: 4, table size: 12
	index: 0, handler: __TI_decompress_rle24
	index: 1, handler: __TI_decompress_none
	index: 2, handler: __TI_zero_init


GLOBAL SYMBOLS: SORTED ALPHABETICALLY BY Name 

address    name
--------   ----
0c077ff0   ALE_Entries_Init
00835458   ALE_entries
0c06cd08   Bus_error_handler
0c081ee0   C$$EXIT
0c081cd8   C$$IO$$
0c06f6d8   C6670_EVM_DDR_Init
0c06e810   C6678_EVM_DDR_Init
00838278   CIC_Regs
0c06d888   CPU_interrupt_enable
0c06d7e0   CPU_interrupt_init
0c0774ec   ConstructPacket
0c06dd48   DDR3_registers_adress_map
008354f8   DDR_REGS_MPAX_cfg_table
0c06e250   DDR_quick_test
0083823c   DestIP
00838236   DestPort
00838058   Dest_MAC_address
0c06eeb0   Dual_Nyquist_EVM_DDR_Init
0c06a8b8   EDMA_CC_error_handler
0c06aacc   EDMA_TC_error_handler
0c069a00   EDMA_TC_priority_cfg
0c069978   EDMA_channel_TC_cfg
0c06a240   EDMA_copy
0c06abf8   EDMA_error_handler
0c06a02c   EDMA_event_disable
0c069fc0   EDMA_event_enable
0c06a458   EDMA_fill
0c069a68   EDMA_init
0c06a108   EDMA_interrupt_disable
0c06a09c   EDMA_interrupt_enable
0c06a178   EDMA_wait
0c06d7b0   EXC_NMI
0c06d6f0   EXC_internal
0c06d7c8   EXC_swgen
0c07a440   Exception_service_routine
00837e50   FDQ_str
0c06dfec   Fill_DDR_ECC_range_by_EDMA
0c072698   Fill_EMAC_header
0c079154   Fill_IP_header
0c079298   Fill_UDP_header
0c078d14   GE_2DSP_Test
0c07b7f4   GE_Check_Free_Queues
0c07ba90   GE_Check_Queue
0c07b990   GE_Check_TxRx_Queues
0c0782f8   GE_DSP0_to_DSP1_test
00838244   GE_INT_TSCL
0c07c270   GE_Interrupts_Init
0c07a138   GE_MISC_MDIO_ISR
0c079e20   GE_Message_ISR
0c07b600   GE_PktDMA_init
0c07b730   GE_QMSS_Accumulation_config
00838248   GE_RX_packet_cnt
008380b0   GE_duplex_str
0c078220   GE_external_loopback_test
0c0781dc   GE_internal_loopback_test
00837fe0   GE_mode_str
0c0779ec   GE_multiple_port_transfer
0c0778f4   GE_signle_port_loopback_test
0c077694   GE_signle_port_transfer
00838078   GE_speed_str
0c0727a4   Get_EMAC_header
0c078cf0   Get_TX_Good_Frames
0c081020   HOSTclose
0c07ffc0   HOSTlseek
0c0803c0   HOSTopen
0c0804a0   HOSTread
0c07f3a0   HOSTrename
0c080ba0   HOSTunlink
0c080c60   HOSTwrite
0c06a820   IDMA_copy
0c06a7f4   IDMA_wait
0c0773a0   InitPayload
0c06cde4   KeyStone_CIC_EXC_handler
0c06c6ec   KeyStone_CIC_exception_events_mapping
0c073410   KeyStone_Copy_FDQ
0c06b104   KeyStone_CorePac_AID_map
0c06e4ec   KeyStone_DDR_ECC_INT_enable
0c06e510   KeyStone_DDR_ECC_init
0c069068   KeyStone_DDR_PLL_init
0c06e704   KeyStone_DDR_clock_phase_init
0c06e354   KeyStone_DDR_full_leveling
0c070420   KeyStone_DDR_init
0c06e7c4   KeyStone_DDR_latch_leveling_configuration
0c06e3ec   KeyStone_DDR_read_incremental_leveling
0c06d228   KeyStone_EXC_external
0c071798   KeyStone_Ethernet_Ports_Init
0c06cb24   KeyStone_Exception_cfg
0c071278   KeyStone_GE_ALE_Init
0c071f24   KeyStone_GE_Accumulate_Statistics
0c071734   KeyStone_GE_CPPI_Src_ID_Init
0c071650   KeyStone_GE_Flow_Control_MAC_Address_Init
0c071db0   KeyStone_GE_Init
0c07150c   KeyStone_GE_Statistics_Init
0c0711b8   KeyStone_GE_soft_reset
0c073008   KeyStone_Host_Descriptor_Queues_init
0c0798e4   KeyStone_HyperLink_Serdes_init
0c071d00   KeyStone_MDIO_Init
0c0728d8   KeyStone_MDIO_PHY_Get_Reg
0c072868   KeyStone_MDIO_PHY_Set_Reg
0c07cab0   KeyStone_MPAX_seg_setup
0c06b914   KeyStone_MPU_MPPA_modify
0c06ba08   KeyStone_MPU_interrupt_enable
0c06bab0   KeyStone_MPU_interrupts_enable
0c06b68c   KeyStone_MPU_range_setup
0c06b70c   KeyStone_MPU_setup
0c06b3c8   KeyStone_MSMC_MP_interrupt_en
0c06b550   KeyStone_MSMC_protection_exception_handler
0c073280   KeyStone_Mono_Descriptor_Queues_init
0c068fd8   KeyStone_PASS_PLL_init
0c068e2c   KeyStone_PLL_init
0c06b18c   KeyStone_PrivID_Remap
0c072c18   KeyStone_QMSS_Descriptor_Regions_init
0c072b48   KeyStone_QMSS_Linking_RAM_init
0c0736a0   KeyStone_Qmss_Config_Acc_Channel
0c0739cc   KeyStone_Qmss_Config_Reclaim_Queue
0c0734d8   KeyStone_Qmss_Download_Firmware
0c073960   KeyStone_Qmss_config_Acc_Timer
0c073894   KeyStone_Qmss_disable_Acc_Channel
0c06b2e8   KeyStone_SES_MPAX_setup
0c06bd74   KeyStone_SL2_EDC_enable
0c06c414   KeyStone_SL2_EDC_handler
0c06be34   KeyStone_SL2_EDC_interrupt_en
0c06b208   KeyStone_SMS_MPAX_setup
0c079644   KeyStone_SRIO_Serdes_init
0c079448   KeyStone_Serdes_PLL_config
0c079d98   KeyStone_Serdes_disable
0c07cc58   KeyStone_XMC_MPAX_setup
0c06dbc0   KeyStone_common_CPU_init
0c06db84   KeyStone_common_device_init
0c0698d8   KeyStone_disable_PSC_Power_Domain
0c06982c   KeyStone_disable_PSC_module
0c0696ec   KeyStone_enable_PSC_module
0c06d9b0   KeyStone_get_device_info
0c06d8c8   KeyStone_get_device_speed_grade
0c0689a4   KeyStone_main_PLL_init
0c06bc90   KeyStone_peripherals_MPU_excepiton_handler
0c06bb94   KeyStone_peripherals_MPU_fault_status
0c073a34   KeyStone_pktDma_Global_Control
0c073a98   KeyStone_pktDma_TxCh_config
0c073af4   KeyStone_pktDma_configureRxFlow
0c079b84   Keystone_SGMII_Serdes_init
0c06ae34   L1D_memory_protection_cfg
0c06c034   L1P_EDC_setup
0c06c2f0   L1P_ED_handler
0c06ada4   L1P_memory_protection_cfg
0c06ad04   L1_MPPA_setup
0c06aec8   L1_cache_protection
008381bc   LL2_EDC_DMA_err_str
008381c0   LL2_EDC_L1D_err_str
008381c4   LL2_EDC_L1P_err_str
0c06c0b8   LL2_EDC_handler
0c06bf50   LL2_EDC_scrub
0c06be8c   LL2_EDC_setup
008381b8   LL2_EDC_victim_err_str
0c06aed8   LL2_MPPA_setup
0c06af74   LL2_Memory_Protection_cfg
0c075768   MemCopy8
0c07580c   MemCopy8Test
0c074dd8   Memory_Address_Bus_Test
0c0746e4   Memory_Address_Test
0c074974   Memory_Data_Bus_Test
0c074830   Memory_Fill_Test
0c0752c8   Memory_error_double_check
0c075238   Memory_quick_test
0c07a7f0   Nested_Exception_service_routine
008380b8   Ns_str
0c07c404   PHY_Link_State_Update
00837ff8   Peri_MPU_err_type_str
0c077df0   Port_OK
00838238   Recv_IP
0c075984   RepeatMemCopy8Test
0c069298   Reset_Timer
00838110   STATS_EN
0c077644   SendPackets
0c0696a8   Service_Watchdog
00838234   SourPort
00838068   Source_MAC_address
0c06fd50   TCI6614_EVM_DDR_Init
0c06b640   TN_MPU5_constant
0c069160   TSC_delay_ms
0c0691f8   TSC_delay_us
0c06914c   TSC_init
0c0692e8   Timer64_Init
00834200   TxDescriptorTempBuffer
0c0773d8   VerifyPacket
0c077478   WaitForRxInterrupt
0c077f20   Wait_PHY_link
00838280   __CIOBUF_
0c0870e0   __TI_CINIT_Base
0c087130   __TI_CINIT_Limit
0c08709c   __TI_Handler_Table_Base
0c0870a8   __TI_Handler_Table_Limit
UNDEFED    __TI_INITARRAY_Base
UNDEFED    __TI_INITARRAY_Limit
00836520   __TI_STACK_END
00001000   __TI_STACK_SIZE
00838114   __TI_STATIC_BASE
00000800   __TI_SYSMEM_SIZE
UNDEFED    __TI_TLS_INIT_Base
UNDEFED    __TI_TLS_INIT_Limit
00000001   __TI_args_main
0c081aa0   __TI_cpp_init
0c081f00   __TI_decompress_none
0c081f20   __TI_decompress_rle24
0083809c   __TI_enable_exit_profile_output
ffffffff   __TI_pprof_out_hndl
ffffffff   __TI_prof_data_size
ffffffff   __TI_prof_data_start
0c080f60   __TI_tls_init
0c080820   __TI_zero_init
ffffffff   __binit__
0c07aa40   __c6xabi_divd
0c07e020   __c6xabi_divf
0c080d20   __c6xabi_divu
0c07f540   __c6xabi_divul
0c07e520   __c6xabi_divull
0c0817a0   __c6xabi_fixdu
0c081820   __c6xabi_fixfu
0c081b00   __c6xabi_frcmpyd_div
0c081d20   __c6xabi_isinf
0c0818a0   __c6xabi_llshl
0c081b60   __c6xabi_llshru
0c081e60   __c6xabi_negll
0c081da0   __c6xabi_strasgi_64plus
ffffffff   __c_args__
0c080d20   __divu
0c081da0   __strasgi_64plus
0c081de0   _args_main
0c0800c0   _auto_init_elf
0c081920   _c_int00
0c0810c0   _cleanup
00838094   _cleanup_ptr
0c07fc60   _closefile
0c085b78   _ctypes_
0c080de0   _doflush
00838098   _dtors_ptr
00837ecc   _ft_end
00837940   _ftable
00838108   _lock
0c0812a0   _minit
0c081e80   _nop
0c07c4c0   _printfi
00835520   _stack
0c081bc0   _subcull
00837140   _sys_memory
00835248   _tmpnams
0083810c   _unlock
0c0801c0   _wrt_ok
0c081ee0   abort
0c084650   acc16_le
0c084010   acc32_le
008353c8   ale_cfg
0c080660   atoi
ffffffff   binit
00837f20   boot_mode_str
00837f40   bus_err_stat_str
0c0690f4   calc_cycle_measure_overhead
0c079348   checksum
0c080740   close
0c0802c0   copy_in
008381b0   cycle_measure_overhead
00837dc8   descMemRegionsCfg
00838040   device_type_str
0c0753a0   edma_Throughput_Test
008380c0   endian_str
0083825c   ethernet_mode
00835388   ethernet_port_cfg
00835488   exception_record
0c080ea0   exit
00837d58   flowCfgTable
00838010   flow_str
0c07ebc0   fputc
0c07cd60   fputs
0c07e2a0   free
00837b20   freeHostQueueCfgTable
0c07fea0   fseek
00837f60   gCIC_EXC_EN_MASK
008381cc   gCIC_EXC_out_num
008381a8   gDSP_Core_Speed_Hz
008381ac   gDSP_board_type
00835424   ge_cfg
0c06ddc0   get_DDR_ECC_ranges
0083811c   gpBootCfgRegs
00838118   gpCGEM_regs
00838130   gpCIC0_regs
00838134   gpCIC1_regs
00838138   gpCIC_regs
008380c8   gpCPSW_port_regs
00838250   gpCPSW_regs
008381a4   gpDDR_regs
0083813c   gpEDMA_CC0_regs
00838140   gpEDMA_CC1_regs
00838144   gpEDMA_CC2_regs
00838088   gpEDMA_CC_regs
00838148   gpEDMA_TC_0_0_regs
0083814c   gpEDMA_TC_0_1_regs
00838150   gpEDMA_TC_1_0_regs
00838154   gpEDMA_TC_1_1_regs
00838158   gpEDMA_TC_1_2_regs
0083815c   gpEDMA_TC_1_3_regs
00838160   gpEDMA_TC_2_0_regs
00838164   gpEDMA_TC_2_1_regs
00838168   gpEDMA_TC_2_2_regs
0083816c   gpEDMA_TC_2_3_regs
00837e80   gpEDMA_TC_regs
0083812c   gpGPIO_regs
008380d0   gpMAC_regs
0083824c   gpMDIO_regs
00838194   gpMPU0_regs
00838198   gpMPU1_regs
0083819c   gpMPU2_regs
008381a0   gpMPU3_regs
00837f80   gpMPU_regs
00838128   gpMSMC_regs
0083821c   gpNetCP_DMA_CfgRegs
00838224   gpNetCP_DMA_RxChCfgRegs
0083822c   gpNetCP_DMA_RxFlowCfgRegs
00838220   gpNetCP_DMA_TxChCfgRegs
00838228   gpNetCP_DMA_TxChPriority
00838254   gpNetCP_regs
00838120   gpPLLC_regs
00838124   gpPSC_regs
008381f4   gpQM_DMA_CfgRegs
008381fc   gpQM_DMA_RxChCfgRegs
00838204   gpQM_DMA_RxFlowCfgRegs
008381f8   gpQM_DMA_TxChCfgRegs
00838200   gpQM_DMA_TxChPriority
008381f0   gpQM_INTD_regs
008380d8   gpQM_PDSP_Cmd
008380e0   gpQM_PDSP_CtrlRegs
008380e8   gpQM_PDSP_IRAM
008381d0   gpQM_configRegs
008381d4   gpQM_descriptorRegions
008381dc   gpQueueManageProxyRegs
008381e4   gpQueueManageProxyVBUSM
008381d8   gpQueueManageRegs
008381e0   gpQueueManageVBUSM
008381e8   gpQueueStatusConfigRegs
008381ec   gpQueueThresholdStatus
008380f0   gpSGMII_regs
00838208   gpSRIO_DMA_CfgRegs
00838210   gpSRIO_DMA_RxChCfgRegs
00838218   gpSRIO_DMA_RxFlowCfgRegs
0083820c   gpSRIO_DMA_TxChCfgRegs
00838214   gpSRIO_DMA_TxChPriority
008380f8   gpStats_regs
00838170   gpTimer0Regs
00838174   gpTimer1Regs
00838178   gpTimer2Regs
0083817c   gpTimer3Regs
00838180   gpTimer4Regs
00838184   gpTimer5Regs
00838188   gpTimer6Regs
0083818c   gpTimer7Regs
00838190   gpTimer8Regs
00837ea8   gpTimerRegs
00838114   gpXMC_regs
00837e10   gstruMpuAddrRange
008381c8   guwIntcCICExcEvtIdx
82340000   hostDescriptor_DDR
00836540   hostDescriptor_LL2
0c085e80   hostDescriptor_SL2
00837ed0   input_clk_str
00837ef8   internal_exception_str
0c07c920   lock_mem_prot_regs
0c081480   lseek
0c080900   ltoa
0c078374   main
0c07f860   malloc
008353ec   mdio_cfg
00835508   mem_prot_key
0c081c20   memccpy
0c081520   memcpy
0c06b430   memory_protection_exception_handler
0c0809e0   memset
00837fa0   message_src_dest
00837fc0   multiPortTest
00838230   numLinkingEntry
82000000   packetBuffer_DDR_Size0
820c0000   packetBuffer_DDR_Size1
00800200   packetBuffer_LL2_Size0
0080c200   packetBuffer_LL2_Size1
0c000000   packetBuffer_SL2_Size0
0c018000   packetBuffer_SL2_Size1
0c07c370   parserRxPacket
00838100   port_connect
0c076d4c   print_GE_MDIO_status
0c076b40   print_GE_ethernet_ports_status
0c075bc0   print_GE_link_ability
0c075c10   print_GE_statistics
0c076da8   print_GE_status_error
0c080ac0   printf
0c081e20   puts
0c0819a0   readmsg
0c081a20   remove
008353f8   serdesLinkSetup
0c07efe0   setvbuf
0083827c   sgmiiSerdesRegs
00834e00   statistics
00838028   test_2DSP_cfg
00838258   test_data_path
00838260   ucTestID
00838274   uiAccPageSize
00838270   uiAccPingPong
00838240   uiGE_MISC_MDIO_INT_num
00838268   uiInitialHostFdqNum
008381b4   uiLL2_scrub_addr
00838264   uiUsedDescRegionNum
0083826c   uiUsedRxFlowNum
00835040   uiaDescriptorAccumulationList
0c081a20   unlink
0c07c9e8   unlock_mem_prot_regs
00800000   vectors
0c081700   write
0c081c80   writemsg


GLOBAL SYMBOLS: SORTED BY Symbol Address 

address    name
--------   ----
00000001   __TI_args_main
00000800   __TI_SYSMEM_SIZE
00001000   __TI_STACK_SIZE
00800000   vectors
00800200   packetBuffer_LL2_Size0
0080c200   packetBuffer_LL2_Size1
00834200   TxDescriptorTempBuffer
00834e00   statistics
00835040   uiaDescriptorAccumulationList
00835248   _tmpnams
00835388   ethernet_port_cfg
008353c8   ale_cfg
008353ec   mdio_cfg
008353f8   serdesLinkSetup
00835424   ge_cfg
00835458   ALE_entries
00835488   exception_record
008354f8   DDR_REGS_MPAX_cfg_table
00835508   mem_prot_key
00835520   _stack
00836520   __TI_STACK_END
00836540   hostDescriptor_LL2
00837140   _sys_memory
00837940   _ftable
00837b20   freeHostQueueCfgTable
00837d58   flowCfgTable
00837dc8   descMemRegionsCfg
00837e10   gstruMpuAddrRange
00837e50   FDQ_str
00837e80   gpEDMA_TC_regs
00837ea8   gpTimerRegs
00837ecc   _ft_end
00837ed0   input_clk_str
00837ef8   internal_exception_str
00837f20   boot_mode_str
00837f40   bus_err_stat_str
00837f60   gCIC_EXC_EN_MASK
00837f80   gpMPU_regs
00837fa0   message_src_dest
00837fc0   multiPortTest
00837fe0   GE_mode_str
00837ff8   Peri_MPU_err_type_str
00838010   flow_str
00838028   test_2DSP_cfg
00838040   device_type_str
00838058   Dest_MAC_address
00838068   Source_MAC_address
00838078   GE_speed_str
00838088   gpEDMA_CC_regs
00838094   _cleanup_ptr
00838098   _dtors_ptr
0083809c   __TI_enable_exit_profile_output
008380b0   GE_duplex_str
008380b8   Ns_str
008380c0   endian_str
008380c8   gpCPSW_port_regs
008380d0   gpMAC_regs
008380d8   gpQM_PDSP_Cmd
008380e0   gpQM_PDSP_CtrlRegs
008380e8   gpQM_PDSP_IRAM
008380f0   gpSGMII_regs
008380f8   gpStats_regs
00838100   port_connect
00838108   _lock
0083810c   _unlock
00838110   STATS_EN
00838114   __TI_STATIC_BASE
00838114   gpXMC_regs
00838118   gpCGEM_regs
0083811c   gpBootCfgRegs
00838120   gpPLLC_regs
00838124   gpPSC_regs
00838128   gpMSMC_regs
0083812c   gpGPIO_regs
00838130   gpCIC0_regs
00838134   gpCIC1_regs
00838138   gpCIC_regs
0083813c   gpEDMA_CC0_regs
00838140   gpEDMA_CC1_regs
00838144   gpEDMA_CC2_regs
00838148   gpEDMA_TC_0_0_regs
0083814c   gpEDMA_TC_0_1_regs
00838150   gpEDMA_TC_1_0_regs
00838154   gpEDMA_TC_1_1_regs
00838158   gpEDMA_TC_1_2_regs
0083815c   gpEDMA_TC_1_3_regs
00838160   gpEDMA_TC_2_0_regs
00838164   gpEDMA_TC_2_1_regs
00838168   gpEDMA_TC_2_2_regs
0083816c   gpEDMA_TC_2_3_regs
00838170   gpTimer0Regs
00838174   gpTimer1Regs
00838178   gpTimer2Regs
0083817c   gpTimer3Regs
00838180   gpTimer4Regs
00838184   gpTimer5Regs
00838188   gpTimer6Regs
0083818c   gpTimer7Regs
00838190   gpTimer8Regs
00838194   gpMPU0_regs
00838198   gpMPU1_regs
0083819c   gpMPU2_regs
008381a0   gpMPU3_regs
008381a4   gpDDR_regs
008381a8   gDSP_Core_Speed_Hz
008381ac   gDSP_board_type
008381b0   cycle_measure_overhead
008381b4   uiLL2_scrub_addr
008381b8   LL2_EDC_victim_err_str
008381bc   LL2_EDC_DMA_err_str
008381c0   LL2_EDC_L1D_err_str
008381c4   LL2_EDC_L1P_err_str
008381c8   guwIntcCICExcEvtIdx
008381cc   gCIC_EXC_out_num
008381d0   gpQM_configRegs
008381d4   gpQM_descriptorRegions
008381d8   gpQueueManageRegs
008381dc   gpQueueManageProxyRegs
008381e0   gpQueueManageVBUSM
008381e4   gpQueueManageProxyVBUSM
008381e8   gpQueueStatusConfigRegs
008381ec   gpQueueThresholdStatus
008381f0   gpQM_INTD_regs
008381f4   gpQM_DMA_CfgRegs
008381f8   gpQM_DMA_TxChCfgRegs
008381fc   gpQM_DMA_RxChCfgRegs
00838200   gpQM_DMA_TxChPriority
00838204   gpQM_DMA_RxFlowCfgRegs
00838208   gpSRIO_DMA_CfgRegs
0083820c   gpSRIO_DMA_TxChCfgRegs
00838210   gpSRIO_DMA_RxChCfgRegs
00838214   gpSRIO_DMA_TxChPriority
00838218   gpSRIO_DMA_RxFlowCfgRegs
0083821c   gpNetCP_DMA_CfgRegs
00838220   gpNetCP_DMA_TxChCfgRegs
00838224   gpNetCP_DMA_RxChCfgRegs
00838228   gpNetCP_DMA_TxChPriority
0083822c   gpNetCP_DMA_RxFlowCfgRegs
00838230   numLinkingEntry
00838234   SourPort
00838236   DestPort
00838238   Recv_IP
0083823c   DestIP
00838240   uiGE_MISC_MDIO_INT_num
00838244   GE_INT_TSCL
00838248   GE_RX_packet_cnt
0083824c   gpMDIO_regs
00838250   gpCPSW_regs
00838254   gpNetCP_regs
00838258   test_data_path
0083825c   ethernet_mode
00838260   ucTestID
00838264   uiUsedDescRegionNum
00838268   uiInitialHostFdqNum
0083826c   uiUsedRxFlowNum
00838270   uiAccPingPong
00838274   uiAccPageSize
00838278   CIC_Regs
0083827c   sgmiiSerdesRegs
00838280   __CIOBUF_
0c000000   packetBuffer_SL2_Size0
0c018000   packetBuffer_SL2_Size1
0c0689a4   KeyStone_main_PLL_init
0c068e2c   KeyStone_PLL_init
0c068fd8   KeyStone_PASS_PLL_init
0c069068   KeyStone_DDR_PLL_init
0c0690f4   calc_cycle_measure_overhead
0c06914c   TSC_init
0c069160   TSC_delay_ms
0c0691f8   TSC_delay_us
0c069298   Reset_Timer
0c0692e8   Timer64_Init
0c0696a8   Service_Watchdog
0c0696ec   KeyStone_enable_PSC_module
0c06982c   KeyStone_disable_PSC_module
0c0698d8   KeyStone_disable_PSC_Power_Domain
0c069978   EDMA_channel_TC_cfg
0c069a00   EDMA_TC_priority_cfg
0c069a68   EDMA_init
0c069fc0   EDMA_event_enable
0c06a02c   EDMA_event_disable
0c06a09c   EDMA_interrupt_enable
0c06a108   EDMA_interrupt_disable
0c06a178   EDMA_wait
0c06a240   EDMA_copy
0c06a458   EDMA_fill
0c06a7f4   IDMA_wait
0c06a820   IDMA_copy
0c06a8b8   EDMA_CC_error_handler
0c06aacc   EDMA_TC_error_handler
0c06abf8   EDMA_error_handler
0c06ad04   L1_MPPA_setup
0c06ada4   L1P_memory_protection_cfg
0c06ae34   L1D_memory_protection_cfg
0c06aec8   L1_cache_protection
0c06aed8   LL2_MPPA_setup
0c06af74   LL2_Memory_Protection_cfg
0c06b104   KeyStone_CorePac_AID_map
0c06b18c   KeyStone_PrivID_Remap
0c06b208   KeyStone_SMS_MPAX_setup
0c06b2e8   KeyStone_SES_MPAX_setup
0c06b3c8   KeyStone_MSMC_MP_interrupt_en
0c06b430   memory_protection_exception_handler
0c06b550   KeyStone_MSMC_protection_exception_handler
0c06b640   TN_MPU5_constant
0c06b68c   KeyStone_MPU_range_setup
0c06b70c   KeyStone_MPU_setup
0c06b914   KeyStone_MPU_MPPA_modify
0c06ba08   KeyStone_MPU_interrupt_enable
0c06bab0   KeyStone_MPU_interrupts_enable
0c06bb94   KeyStone_peripherals_MPU_fault_status
0c06bc90   KeyStone_peripherals_MPU_excepiton_handler
0c06bd74   KeyStone_SL2_EDC_enable
0c06be34   KeyStone_SL2_EDC_interrupt_en
0c06be8c   LL2_EDC_setup
0c06bf50   LL2_EDC_scrub
0c06c034   L1P_EDC_setup
0c06c0b8   LL2_EDC_handler
0c06c2f0   L1P_ED_handler
0c06c414   KeyStone_SL2_EDC_handler
0c06c6ec   KeyStone_CIC_exception_events_mapping
0c06cb24   KeyStone_Exception_cfg
0c06cd08   Bus_error_handler
0c06cde4   KeyStone_CIC_EXC_handler
0c06d228   KeyStone_EXC_external
0c06d6f0   EXC_internal
0c06d7b0   EXC_NMI
0c06d7c8   EXC_swgen
0c06d7e0   CPU_interrupt_init
0c06d888   CPU_interrupt_enable
0c06d8c8   KeyStone_get_device_speed_grade
0c06d9b0   KeyStone_get_device_info
0c06db84   KeyStone_common_device_init
0c06dbc0   KeyStone_common_CPU_init
0c06dd48   DDR3_registers_adress_map
0c06ddc0   get_DDR_ECC_ranges
0c06dfec   Fill_DDR_ECC_range_by_EDMA
0c06e250   DDR_quick_test
0c06e354   KeyStone_DDR_full_leveling
0c06e3ec   KeyStone_DDR_read_incremental_leveling
0c06e4ec   KeyStone_DDR_ECC_INT_enable
0c06e510   KeyStone_DDR_ECC_init
0c06e704   KeyStone_DDR_clock_phase_init
0c06e7c4   KeyStone_DDR_latch_leveling_configuration
0c06e810   C6678_EVM_DDR_Init
0c06eeb0   Dual_Nyquist_EVM_DDR_Init
0c06f6d8   C6670_EVM_DDR_Init
0c06fd50   TCI6614_EVM_DDR_Init
0c070420   KeyStone_DDR_init
0c0711b8   KeyStone_GE_soft_reset
0c071278   KeyStone_GE_ALE_Init
0c07150c   KeyStone_GE_Statistics_Init
0c071650   KeyStone_GE_Flow_Control_MAC_Address_Init
0c071734   KeyStone_GE_CPPI_Src_ID_Init
0c071798   KeyStone_Ethernet_Ports_Init
0c071d00   KeyStone_MDIO_Init
0c071db0   KeyStone_GE_Init
0c071f24   KeyStone_GE_Accumulate_Statistics
0c072698   Fill_EMAC_header
0c0727a4   Get_EMAC_header
0c072868   KeyStone_MDIO_PHY_Set_Reg
0c0728d8   KeyStone_MDIO_PHY_Get_Reg
0c072b48   KeyStone_QMSS_Linking_RAM_init
0c072c18   KeyStone_QMSS_Descriptor_Regions_init
0c073008   KeyStone_Host_Descriptor_Queues_init
0c073280   KeyStone_Mono_Descriptor_Queues_init
0c073410   KeyStone_Copy_FDQ
0c0734d8   KeyStone_Qmss_Download_Firmware
0c0736a0   KeyStone_Qmss_Config_Acc_Channel
0c073894   KeyStone_Qmss_disable_Acc_Channel
0c073960   KeyStone_Qmss_config_Acc_Timer
0c0739cc   KeyStone_Qmss_Config_Reclaim_Queue
0c073a34   KeyStone_pktDma_Global_Control
0c073a98   KeyStone_pktDma_TxCh_config
0c073af4   KeyStone_pktDma_configureRxFlow
0c0746e4   Memory_Address_Test
0c074830   Memory_Fill_Test
0c074974   Memory_Data_Bus_Test
0c074dd8   Memory_Address_Bus_Test
0c075238   Memory_quick_test
0c0752c8   Memory_error_double_check
0c0753a0   edma_Throughput_Test
0c075768   MemCopy8
0c07580c   MemCopy8Test
0c075984   RepeatMemCopy8Test
0c075bc0   print_GE_link_ability
0c075c10   print_GE_statistics
0c076b40   print_GE_ethernet_ports_status
0c076d4c   print_GE_MDIO_status
0c076da8   print_GE_status_error
0c0773a0   InitPayload
0c0773d8   VerifyPacket
0c077478   WaitForRxInterrupt
0c0774ec   ConstructPacket
0c077644   SendPackets
0c077694   GE_signle_port_transfer
0c0778f4   GE_signle_port_loopback_test
0c0779ec   GE_multiple_port_transfer
0c077df0   Port_OK
0c077f20   Wait_PHY_link
0c077ff0   ALE_Entries_Init
0c0781dc   GE_internal_loopback_test
0c078220   GE_external_loopback_test
0c0782f8   GE_DSP0_to_DSP1_test
0c078374   main
0c078cf0   Get_TX_Good_Frames
0c078d14   GE_2DSP_Test
0c079154   Fill_IP_header
0c079298   Fill_UDP_header
0c079348   checksum
0c079448   KeyStone_Serdes_PLL_config
0c079644   KeyStone_SRIO_Serdes_init
0c0798e4   KeyStone_HyperLink_Serdes_init
0c079b84   Keystone_SGMII_Serdes_init
0c079d98   KeyStone_Serdes_disable
0c079e20   GE_Message_ISR
0c07a138   GE_MISC_MDIO_ISR
0c07a440   Exception_service_routine
0c07a7f0   Nested_Exception_service_routine
0c07aa40   __c6xabi_divd
0c07b600   GE_PktDMA_init
0c07b730   GE_QMSS_Accumulation_config
0c07b7f4   GE_Check_Free_Queues
0c07b990   GE_Check_TxRx_Queues
0c07ba90   GE_Check_Queue
0c07c270   GE_Interrupts_Init
0c07c370   parserRxPacket
0c07c404   PHY_Link_State_Update
0c07c4c0   _printfi
0c07c920   lock_mem_prot_regs
0c07c9e8   unlock_mem_prot_regs
0c07cab0   KeyStone_MPAX_seg_setup
0c07cc58   KeyStone_XMC_MPAX_setup
0c07cd60   fputs
0c07e020   __c6xabi_divf
0c07e2a0   free
0c07e520   __c6xabi_divull
0c07ebc0   fputc
0c07efe0   setvbuf
0c07f3a0   HOSTrename
0c07f540   __c6xabi_divul
0c07f860   malloc
0c07fc60   _closefile
0c07fea0   fseek
0c07ffc0   HOSTlseek
0c0800c0   _auto_init_elf
0c0801c0   _wrt_ok
0c0802c0   copy_in
0c0803c0   HOSTopen
0c0804a0   HOSTread
0c080660   atoi
0c080740   close
0c080820   __TI_zero_init
0c080900   ltoa
0c0809e0   memset
0c080ac0   printf
0c080ba0   HOSTunlink
0c080c60   HOSTwrite
0c080d20   __c6xabi_divu
0c080d20   __divu
0c080de0   _doflush
0c080ea0   exit
0c080f60   __TI_tls_init
0c081020   HOSTclose
0c0810c0   _cleanup
0c0812a0   _minit
0c081480   lseek
0c081520   memcpy
0c081700   write
0c0817a0   __c6xabi_fixdu
0c081820   __c6xabi_fixfu
0c0818a0   __c6xabi_llshl
0c081920   _c_int00
0c0819a0   readmsg
0c081a20   remove
0c081a20   unlink
0c081aa0   __TI_cpp_init
0c081b00   __c6xabi_frcmpyd_div
0c081b60   __c6xabi_llshru
0c081bc0   _subcull
0c081c20   memccpy
0c081c80   writemsg
0c081cd8   C$$IO$$
0c081d20   __c6xabi_isinf
0c081da0   __c6xabi_strasgi_64plus
0c081da0   __strasgi_64plus
0c081de0   _args_main
0c081e20   puts
0c081e60   __c6xabi_negll
0c081e80   _nop
0c081ee0   C$$EXIT
0c081ee0   abort
0c081f00   __TI_decompress_none
0c081f20   __TI_decompress_rle24
0c084010   acc32_le
0c084650   acc16_le
0c085b78   _ctypes_
0c085e80   hostDescriptor_SL2
0c08709c   __TI_Handler_Table_Base
0c0870a8   __TI_Handler_Table_Limit
0c0870e0   __TI_CINIT_Base
0c087130   __TI_CINIT_Limit
82000000   packetBuffer_DDR_Size0
820c0000   packetBuffer_DDR_Size1
82340000   hostDescriptor_DDR
ffffffff   __TI_pprof_out_hndl
ffffffff   __TI_prof_data_size
ffffffff   __TI_prof_data_start
ffffffff   __binit__
ffffffff   __c_args__
ffffffff   binit
UNDEFED    __TI_INITARRAY_Base
UNDEFED    __TI_INITARRAY_Limit
UNDEFED    __TI_TLS_INIT_Base
UNDEFED    __TI_TLS_INIT_Limit

[415 symbols]
